:1000000010C01FC01EC01DC01CC01BC01AC019C01C
:1000100018C017C016C01CC014C013C012C011C035
:1000200010C011241FBECFE5D2E0DEBFCDBF10E06F
:10003000A0E6B0E001C01D92A936B107E1F704D0F7
:1000400063C0DECF089508954CD0FCDFFCDFFECF07
:100050001F920F920FB60F9211242F933F938F93FD
:100060009F93AF93BF938091640090916500A0919E
:100070006600B091670030916800232F2D5F2D3707
:1000800028F02D570296A11DB11D03C00196A11D98
:10009000B11D209368008093640090936500A09345
:1000A0006600B09367008091600090916100A0911C
:1000B0006200B09163000196A11DB11D80936000A4
:1000C00090936100A0936200B0936300BF91AF91E1
:1000D0009F918F913F912F910F900FBE0F901F9086
:1000E0001895789480B7836080BF83B7877F83BF7C
:1000F00083B7887F836083BF89B7816089BF86B1FA
:0C010000876086B9379A0895F894FFCF05
:00000001FF
